:100000000C943E001895000018950000189500000B
:10001000189500001895000018950000189500002C
:10002000189500001895000018950000189500001C
:10003000189500001895000018950000189500000C
:1000400018950000189500001895000018950000FC
:1000500018950000189500001895000018950000EC
:1000600018950000189500001895000018950000DC
:100070001895000018950000189500008FEF8DBFAF
:10008000C0EEE0ED4E2E80E18EBFD0E1F0E15F2EBC
:10009000EEEFFFE0A0E0B1E0A89584B7082E877FDF
:1000A00084BF88E19927809360009093600088273F
:1000B0008D933197E9F787E08093C40080E08093C7
:1000C000C50088E18093C100662487E880937A00A8
:1000D00080E080937C003B9A219A3C9A3A9A399A24
:1000E000549A3D9A389A539A209A559A3F9A239A4D
:1000F000099A3E9A0D9A229A579A569A02E518EB57
:100100002EE135E0A8E0B1E00D931D932D933C93D3
:1001100081E08093000184E08093010183E080937B
:10012000140180E08093020185E0809303012A9A04
:10013000E1E0F0E00E944013459AE1E0F0E00E9427
:100140004013409844985C985B9A2998479A2B9A58
:100150001198449A81E090E00E94A61344983A9A3C
:100160003B9A4398A0E0B1E0119698E08E919830C8
:1001700018F4392F992702C038E09850881F429808
:1001800008F4429A00000000439AEF93FF93EFE0D7
:10019000F0E00E949D13FF91EF914398EF93FF933E
:1001A000EFE0F0E00E949D13FF91EF913A9531F757
:1001B0009923E1F683ED809311013A9A3B9A439893
:1001C000A1E1B1E0119698E08E91983018F4392FA2
:1001D000992702C038E09850881F429808F4429A44
:1001E00000000000439AEF93FF93E6E4F0E00E94E2
:1001F0009D13FF91EF914398EF93FF93E6E4F0E0B6
:100200000E949D13FF91EF913A9531F79923E1F602
:1002100080E0809311013A9A3B9A4398A1E1B1E0C2
:10022000119698E08E91983018F4392F992702C0D2
:1002300038E09850881F429808F4429A0000000065
:10024000439AEF93FF93E6E4F0E00E949D13FF9141
:10025000EF914398EF93FF93E6E4F0E00E949D1343
:10026000FF91EF913A9531F79923E1F680E280937F
:1002700011013A9A3B9A4398A1E1B1E0119698E0B6
:100280008E91983018F4392F992702C038E0985091
:10029000881F429808F4429A00000000439AEF93A6
:1002A000FF93E6E4F0E00E949D13FF91EF914398E5
:1002B000EF93FF93E6E4F0E00E949D13FF91EF912E
:1002C0003A9531F79923E1F6419A419870917A0075
:1002D000706870937A005C9A01E010E020E030E0F2
:1002E000AAE1B1E00D931D932D933C9300917C0006
:1002F000007E066000937C000E94D813A7E9B4E05A
:100300008D939C93A7E9B4E00D911C91003951E0C5
:10031000150718F011F00C948F010C9494015C985F
:100320001598479A0C9498015C9A159A4798469AA2
:100330000E944814A0E3B1E035E00E940A130E9435
:100340004514A0E3B1E00E941614A6E5B1E00D93B8
:100350001C93A6E5B1E00D911C91023050E0150709
:1003600011F00C94B7010E94C50B0C940E020030E2
:1003700050E0150711F00C94C1010E9459020C9431
:100380000E02013050E0150711F00C94CB010E94D1
:1003900059020C940E02033050E0150711F00C9432
:1003A000D5010E9459020C940E02043050E015074A
:1003B00011F00C94DF010E9459020C940E020630D9
:1003C00050E0150711F00C94E9010E9410020C9402
:1003D0000E02083050E0150711F00C940202009153
:1003E0007C00007E076000937C000E94D813A7E980
:1003F000B4E08D939C9332E0A7E9B4E00E943113FE
:100400000C940E02093050E0150711F00C940E0206
:10041000E6E9F8E20E942A130E9436130C94760152
:100420000E944814AEE1B1E035E00E940A130E9438
:100430004514AEE1B1E00E941614AAE1B1E00D93BB
:100440001D932D933D9308950AE010E020E030E0E5
:10045000AAE1B1E04D915D916D917C910E94B5133F
:10046000ACE8B4E00D931D932D933D9301E010E0B3
:1004700020E030E0A8E8B4E00D931D932D933C9369
:10048000ACE8B4E04D915D916D917C91A8E8B4E049
:100490000D911D912D913C910E9403141CF011F0BF
:1004A0000C945802A8E8B4E00E94F9120C9440029F
:1004B00008950E944814A6E3B1E03FE00E940A13A9
:1004C0000E9445140E944814A4E2B1E035E00E9465
:1004D0000A130E9445140E944814AAE2B1E035E0D4
:1004E0000E940A130E9445140E944814A6E4B1E039
:1004F0003FE00E940A130E944514449A81E090E074
:100500000E94A61344983A9A3B9A4398A0E0B1E01F
:10051000119698E08E91983018F4392F992702C0DF
:1005200038E09850881F429808F4429A0000000072
:10053000439AEF93FF93EFE0F0E00E949D13FF9149
:10054000EF914398EF93FF93EFE0F0E00E949D134B
:10055000FF91EF913A9531F79923E1F683ED80937E
:1005600011013A9A3B9A4398A1E1B1E0119698E0C3
:100570008E91983018F4392F992702C038E098509E
:10058000881F429808F4429A00000000439AEF93B3
:10059000FF93E6E4F0E00E949D13FF91EF914398F2
:1005A000EF93FF93E6E4F0E00E949D13FF91EF913B
:1005B0003A9531F79923E1F680E0809311013A9A58
:1005C0003B9A4398A1E1B1E0119698E08E91983062
:1005D00018F4392F992702C038E09850881F4298A4
:1005E00008F4429A00000000439AEF93FF93E6E478
:1005F000F0E00E949D13FF91EF914398EF93FF93DA
:10060000E6E4F0E00E949D13FF91EF913A9531F7F7
:100610009923E1F680E0809311013A9A3B9A43983E
:10062000A1E1B1E0119698E08E91983018F4392F3D
:10063000992702C038E09850881F429808F4429ADF
:1006400000000000439AEF93FF93E6E4F0E00E947D
:100650009D13FF91EF914398EF93FF93E6E4F0E051
:100660000E949D13FF91EF913A9531F79923E1F69E
:10067000419A41983A9A3B9A4398A2E0B1E0119688
:1006800098E08E91983018F4392F992702C038E0FD
:100690009850881F429808F4429A00000000439A3C
:1006A000EF93FF93E6E4F0E00E949D13FF91EF913A
:1006B0004398EF93FF93E6E4F0E00E949D13FF91CF
:1006C000EF913A9531F79923E1F680E480930C019C
:1006D0003A9A3B9A4398ACE0B1E0119698E08E913B
:1006E000983018F4392F992702C038E09850881FA5
:1006F000429808F4429A00000000439AEF93FF9357
:10070000E6E4F0E00E949D13FF91EF914398EF9390
:10071000FF93E6E4F0E00E949D13FF91EF913A957C
:1007200031F79923E1F63A9A3B9A4398A4E1B1E074
:10073000119698E08E91983018F4392F992702C0BD
:1007400038E09850881F429808F4429A0000000050
:10075000439AEF93FF93E6E4F0E00E949D13FF912C
:10076000EF914398EF93FF93E6E4F0E00E949D132E
:10077000FF91EF913A9531F79923E1F680E080936C
:1007800015013A9A3B9A4398A5E1B1E0119698E099
:100790008E91983018F4392F992702C038E098507C
:1007A000881F429808F4429A00000000439AEF9391
:1007B000FF93E6E4F0E00E949D13FF91EF914398D0
:1007C000EF93FF93E6E4F0E00E949D13FF91EF9119
:1007D0003A9531F79923E1F683E0809315013A9A2F
:1007E0003B9A4398A5E1B1E0119698E08E9198303C
:1007F00018F4392F992702C038E09850881F429882
:1008000008F4429A00000000439AEF93FF93E6E455
:10081000F0E00E949D13FF91EF914398EF93FF93B7
:10082000E6E4F0E00E949D13FF91EF913A9531F7D5
:100830009923E1F680E0809315013A9A3B9A439818
:10084000A5E1B1E0119698E08E91983018F4392F17
:10085000992702C038E09850881F429808F4429ABD
:1008600000000000439AEF93FF93E6E4F0E00E945B
:100870009D13FF91EF914398EF93FF93E6E4F0E02F
:100880000E949D13FF91EF913A9531F79923E1F67C
:100890003A9A3B9A4398A2E0B1E0119698E08E9183
:1008A000983018F4392F992702C038E09850881FE3
:1008B000429808F4429A00000000439AEF93FF9395
:1008C000E6E4F0E00E949D13FF91EF914398EF93CF
:1008D000FF93E6E4F0E00E949D13FF91EF913A95BB
:1008E00031F79923E1F680E880930C013A9A3B9A1C
:1008F0004398ACE0B1E0119698E08E91983018F4EE
:10090000392F992702C038E09850881F429808F480
:10091000429A00000000439AEF93FF93E6E4F0E070
:100920000E949D13FF91EF914398EF93FF93E6E4AC
:10093000F0E00E949D13FF91EF913A9531F79923D2
:10094000E1F63A9A3B9A4398A4E1B1E0119698E017
:100950008E91983018F4392F992702C038E09850BA
:10096000881F429808F4429A00000000439AEF93CF
:10097000FF93E6E4F0E00E949D13FF91EF9143980E
:10098000EF93FF93E6E4F0E00E949D13FF91EF9157
:100990003A9531F79923E1F680E0809315013A9A70
:1009A0003B9A4398A5E1B1E0119698E08E9198307A
:1009B00018F4392F992702C038E09850881F4298C0
:1009C00008F4429A00000000439AEF93FF93E6E494
:1009D000F0E00E949D13FF91EF914398EF93FF93F6
:1009E000E6E4F0E00E949D13FF91EF913A9531F714
:1009F0009923E1F681E0809315013A9A3B9A439856
:100A0000A5E1B1E0119698E08E91983018F4392F55
:100A1000992702C038E09850881F429808F4429AFB
:100A200000000000439AEF93FF93E6E4F0E00E9499
:100A30009D13FF91EF914398EF93FF93E6E4F0E06D
:100A40000E949D13FF91EF913A9531F79923E1F6BA
:100A500080E0809315013A9A3B9A4398A5E1B1E072
:100A6000119698E08E91983018F4392F992702C08A
:100A700038E09850881F429808F4429A000000001D
:100A8000439AEF93FF93E6E4F0E00E949D13FF91F9
:100A9000EF914398EF93FF93E6E4F0E00E949D13FB
:100AA000FF91EF913A9531F79923E1F6419A4198F8
:100AB000A6E3B1E00E941614ACE5B1E00D931D93DE
:100AC0002D933D93A4E2B1E00E941614ADE0B1E095
:100AD0000D931C93AAE2B1E00E941614A8E5B1E0C0
:100AE0000D931D932D933D93A6E4B1E00E9416143F
:100AF000A0E6B1E00D931D932D933D93A4E9B4E0DE
:100B00000E941614A7E9B4E00D931C93A6E5B1E08A
:100B10000D911C91003050E0150781E009F080E054
:100B20008F93A6E5B1E00D911C91033050E01507BD
:100B300081E009F080E09F91892B8F93A6E5B1E0D9
:100B40000D911C91043050E0150781E009F080E020
:100B50009F91892B882311F40C94B2055D982898F5
:100B60005B9A2998A6E5B1E00D911C91013050E007
:100B7000150711F00C94C0055D9A28985B98299888
:100B8000A8E5B1E00D911D912D913C9144E650E016
:100B900060E070E00E944913A6E1B1E04D935D93DF
:100BA0006D937D9381E08093990481E08093990413
:100BB000A6E1B1E04D915D916D917C91A9E9B4E020
:100BC0000C911127222733270E9403141CF011F0E7
:100BD0000C94F4050E94F605A9E9B4E08C918F5FAE
:100BE0008C9310F40C94D805449A08954498159861
:100BF00085E090E00E94A61301E010E020E030E0E4
:100C0000A4E6B1E00D931D932D933C9344E650E090
:100C100060E070E0A4E6B1E00D911D912D913C9152
:100C20000E9403141CF011F00C94720B3A9A3B9A38
:100C30004398A2E0B1E0119698E08E91983018F4B4
:100C4000392F992702C038E09850881F429808F43D
:100C5000429A00000000439A000000004398000000
:100C600000003A9591F7992341F780EC80930C01AD
:100C70003A9A3B9A4398ACE0B1E0119698E08E9195
:100C8000983018F4392F992702C038E09850881FFF
:100C9000429808F4429A00000000439A00000000C5
:100CA0004398000000003A9591F7992341F73A9A4A
:100CB0003B9A4398A1E0B1E0119698E08E9198306C
:100CC00018F4392F992702C038E09850881F4298AD
:100CD00008F4429A00000000439A00000000439884
:100CE000000000003A9591F7992341F73A9A3B9A10
:100CF0004398ACE5B1E0149690E28E91983018F4E8
:100D0000392F992702C038E09850881F429808F47C
:100D1000429A00000000439A00000000439800003F
:100D200000003A9591F7992341F73A9A3B9A4398F4
:100D3000A3E0B1E0119698E08E91983018F4392F25
:100D4000992702C038E09850881F429808F4429AC8
:100D500000000000439A00000000439800000000DB
:100D60003A9591F7992341F780E090E0ADE0B1E04A
:100D70008D939C933A9A3B9A4398ADE0B1E01296DA
:100D800090E18E91983018F4392F992702C038E0FD
:100D90009850881F429808F4429A00000000439A35
:100DA000000000004398000000003A9591F7992355
:100DB00041F7419A41980E942402A6E5B1E00D91C5
:100DC0001C91013050E0150711F00C9447072A9848
:100DD0002A9A2A9884EB94EFA2E1B1E08D939C9338
:100DE00080E090E0A4E6B1E0AD90BC90A6E6B1E072
:100DF000AA0CBB1CAA0DBB1D8D939C93569A579AA7
:100E00005F98A2E1B1E012969EE08E91983018F4BE
:100E1000392F992702C038E09850881F5E9808F44F
:100E20005E9A000000005F9A000000005F980000DA
:100E300000003A9591F7992341F72A9A2A98579AF0
:100E400052985F9A90E1A4E6B1E0AD90BC90A6E61E
:100E5000B1E0AA0CBB1CAA0DBB1D1296983018F469
:100E6000392F992702C038E098505F9800000000A1
:100E700088944A990894881F5F9A000000003A9568
:100E8000A1F78E93992351F72A9A0C9495072A98E3
:100E900084EB90EFA2E1B1E08D939C93569A579A20
:100EA0005F98A2E1B1E012969EE08E91983018F41E
:100EB000392F992702C038E09850881F5E9808F4AF
:100EC0005E9A000000005F9A000000005F9800003A
:100ED00000003A9591F7992341F72A9A2A98579A50
:100EE00052985F9A90E1A4E6B1E0AD90BC90A6E67E
:100EF000B1E0AA0CBB1CAA0DBB1D1296983018F4C9
:100F0000392F992702C038E098505F980000000000
:100F100088944A990894881F5F9A000000003A95C7
:100F2000A1F78E93992351F72A9A3A9A3B9A4398BC
:100F3000A2E0B1E0119698E08E91983018F4392F24
:100F4000992702C038E09850881F429808F4429AC6
:100F500000000000439A00000000439800000000D9
:100F60003A9591F7992341F780E480930C013A9ADE
:100F70003B9A4398ACE0B1E0119698E08E9198309E
:100F800018F4392F992702C038E09850881F4298EA
:100F900008F4429A00000000439A000000004398C1
:100FA000000000003A9591F7992341F73A9A3B9A4D
:100FB0004398A3E0B1E0119698E08E91983018F430
:100FC000392F992702C038E09850881F429808F4BA
:100FD000429A00000000439A00000000439800007D
:100FE00000003A9591F7992341F780E090E1ADE058
:100FF000B1E08D939C933A9A3B9A4398ADE0B1E06F
:10100000129690E18E91983018F4392F992702C0EA
:1010100038E09850881F429808F4429A0000000077
:10102000439A000000004398000000003A9591F7B1
:10103000992341F7419A41980E942402A6E5B1E024
:101040000D911C91013050E0150711F00C948808A7
:1010500084EB94EFA2E1B1E08D939C9380E090E06B
:10106000A4E6B1E0AD90BC90AEE2B2E0AA0CBB1C2D
:10107000AA0DBB1D8D939C932A982A9A2A98569A5A
:10108000579A5F98A2E1B1E012969EE08E91983057
:1010900018F4392F992702C038E09850881F5E98BD
:1010A00008F45E9A000000005F9A000000005F985C
:1010B000000000003A9591F7992341F72A9A2A985F
:1010C000579A52985F9A90E1A4E6B1E0AD90BC9037
:1010D000AEE2B2E0AA0CBB1CAA0DBB1D1296983062
:1010E00018F4392F992702C038E098505F98000013
:1010F000000088944A990894881F5F9A00000000B5
:101100003A95A1F78E93992351F72A9A0C94D60811
:101110002A9884EB90EFA2E1B1E08D939C93569ACC
:10112000579A5F98A2E1B1E012969EE08E919830B6
:1011300018F4392F992702C038E09850881F5E981C
:1011400008F45E9A000000005F9A000000005F98BB
:10115000000000003A9591F7992341F72A9A2A98BE
:10116000579A52985F9A90E1A4E6B1E0AD90BC9096
:10117000AEE2B2E0AA0CBB1CAA0DBB1D12969830C1
:1011800018F4392F992702C038E098505F98000072
:10119000000088944A990894881F5F9A0000000014
:1011A0003A95A1F78E93992351F72A9A3A9A3B9A46
:1011B0004398A2E0B1E0119698E08E91983018F42F
:1011C000392F992702C038E09850881F429808F4B8
:1011D000429A00000000439A00000000439800007B
:1011E00000003A9591F7992341F780E480930C0130
:1011F0003A9A3B9A4398ACE0B1E0119698E08E9110
:10120000983018F4392F992702C038E09850881F79
:10121000429808F4429A00000000439A000000003F
:101220004398000000003A9591F7992341F73A9AC4
:101230003B9A4398A3E0B1E0119698E08E919830E4
:1012400018F4392F992702C038E09850881F429827
:1012500008F4429A00000000439A000000004398FE
:10126000000000003A9591F7992341F780E090E261
:10127000ADE0B1E08D939C933A9A3B9A4398ADE0F0
:10128000B1E0129690E18E91983018F4392F992799
:1012900002C038E09850881F429808F4429A000033
:1012A0000000439A000000004398000000003A95B7
:1012B00091F7992341F7419A41980E942402A6E5AB
:1012C000B1E00D911C91013050E0150711F00C9424
:1012D000C90984EB94EFA2E1B1E08D939C9380E087
:1012E00090E0A4E6B1E0AD90BC90A6EFB2E0AA0C0D
:1012F000BB1CAA0DBB1D8D939C932A982A9A2A98F1
:10130000569A579A5F98A2E1B1E012969EE08E91AC
:10131000983018F4392F992702C038E09850881F68
:101320005E9808F45E9A000000005F9A00000000DA
:101330005F98000000003A9591F7992341F72A9AA7
:101340002A98579A52985F9A90E1A4E6B1E0AD903E
:10135000BC90A6EFB2E0AA0CBB1CAA0DBB1D129656
:10136000983018F4392F992702C038E098505F98C8
:101370000000000088944A990894881F5F9A000032
:1013800000003A95A1F78E93992351F72A9A0C946D
:10139000170A2A9884EB90EFA2E1B1E08D939C9319
:1013A000569A579A5F98A2E1B1E012969EE08E910C
:1013B000983018F4392F992702C038E09850881FC8
:1013C0005E9808F45E9A000000005F9A000000003A
:1013D0005F98000000003A9591F7992341F72A9A07
:1013E0002A98579A52985F9A90E1A4E6B1E0AD909E
:1013F000BC90A6EFB2E0AA0CBB1CAA0DBB1D1296B6
:10140000983018F4392F992702C038E098505F9827
:101410000000000088944A990894881F5F9A000091
:1014200000003A95A1F78E93992351F72A9A3A9A98
:101430003B9A4398A2E0B1E0119698E08E919830E3
:1014400018F4392F992702C038E09850881F429825
:1014500008F4429A00000000439A000000004398FC
:10146000000000003A9591F7992341F780E48093BA
:101470000C013A9A3B9A4398ACE0B1E0119698E09F
:101480008E91983018F4392F992702C038E098507F
:10149000881F429808F4429A00000000439A000016
:1014A00000004398000000003A9591F7992341F716
:1014B0003A9A3B9A4398A3E0B1E0119698E08E9156
:1014C000983018F4392F992702C038E09850881FB7
:1014D000429808F4429A00000000439A000000007D
:1014E0004398000000003A9591F7992341F780E076
:1014F00090E3ADE0B1E08D939C933A9A3B9A439888
:10150000ADE0B1E0129690E18E91983018F4392F49
:10151000992702C038E09850881F429808F4429AF0
:1015200000000000439A0000000043980000000003
:101530003A9591F7992341F7419A41980E942402E4
:10154000A6E5B1E00D911C91013050E0150711F0B6
:101550000C940A0B84EB94EFA2E1B1E08D939C9381
:1015600080E090E0A4E6B1E0AD90BC90AEEBB3E0DB
:10157000AA0CBB1CAA0DBB1D8D939C932A982A9A7A
:101580002A98569A579A5F98A2E1B1E012969EE087
:101590008E91983018F4392F992702C038E098506E
:1015A000881F5E9808F45E9A000000005F9A0000B1
:1015B00000005F98000000003A9591F7992341F7E9
:1015C0002A9A2A98579A52985F9A90E1A4E6B1E035
:1015D000AD90BC90AEEBB3E0AA0CBB1CAA0DBB1D3A
:1015E0001296983018F4392F992702C038E0985095
:1015F0005F980000000088944A990894881F5F9AB9
:10160000000000003A95A1F78E93992351F72A9A8A
:101610000C94580B2A9884EB90EFA2E1B1E08D93E3
:101620009C93569A579A5F98A2E1B1E012969EE079
:101630008E91983018F4392F992702C038E09850CD
:10164000881F5E9808F45E9A000000005F9A000010
:1016500000005F98000000003A9591F7992341F748
:101660002A9A2A98579A52985F9A90E1A4E6B1E094
:10167000AD90BC90AEEBB3E0AA0CBB1CAA0DBB1D99
:101680001296983018F4392F992702C038E09850F4
:101690005F980000000088944A990894881F5F9A18
:1016A000000000003A95A1F78E93992351F72A9AEA
:1016B000ACE5B1E00D911D912D913C91A0E6B1E01A
:1016C0004D915D916D917C910E94FE13ACE5B1E06E
:1016D0000D931D932D933D93A4E6B1E00E94F91262
:1016E0000C940606159A81E090E00E94A61381E012
:1016F00080939A0481E080939A0400919A040436BE
:1017000018F011F00C94C00B32E0AAE9B4E0AD90EF
:10171000BB24A6E6B1E0AA0CBB1CAA0DBB1D0E940F
:10172000311332E0AAE9B4E0AD90BB24AEE2B2E0FE
:10173000AA0CBB1CAA0DBB1D0E94311332E0AAE902
:10174000B4E0AD90BB24A6EFB2E0AA0CBB1CAA0D7E
:10175000BB1D0E94311332E0AAE9B4E0AD90BB2476
:10176000AEEBB3E0AA0CBB1CAA0DBB1D0E9431134B
:10177000AAE9B4E08C918F5F8C9310F40C947D0BEC
:1017800084E190E00E94A613089544980E944814B2
:10179000ABE9B4E03FE00E940A130E9445140E94A6
:1017A0004814ABEAB4E03FE00E940A130E944514DB
:1017B0000E944814ABEBB4E036E00E940A130E948A
:1017C00045140E944814A2ECB4E035E00E940A13CC
:1017D0000E9445140E944814A8ECB4E036E00E9430
:1017E0000A130E9445140E944814AFECB4E036E09E
:1017F0000E940A130E944514ABE9B4E00E9416143B
:10180000A6EDB4E00D931D932D933D93ABEAB4E0A8
:101810000E941614AAEDB4E00D931D932D933D93F1
:10182000ABEBB4E00E941614AEEDB4E00D931C9344
:10183000A2ECB4E00E941614A0EEB4E00C93A8EC65
:10184000B4E00E941614A1EEB4E00D931C93AFEC2B
:10185000B4E00E941614A3EEB4E00D931C935D98BF
:10186000289A5B9A299A449A81E090E00E94A613F4
:1018700044983A9A3B9A4398A0E0B1E0119698E0D8
:101880008E91983018F4392F992702C038E098507B
:10189000881F429808F4429A00000000439AEF9390
:1018A000FF93EFE0F0E00E949D13FF91EF914398CA
:1018B000EF93FF93EFE0F0E00E949D13FF91EF9113
:1018C0003A9531F79923E1F683ED809311013A9A25
:1018D0003B9A4398A1E1B1E0119698E08E9198303F
:1018E00018F4392F992702C038E09850881F429881
:1018F00008F4429A00000000439AEF93FF93E6E455
:10190000F0E00E949D13FF91EF914398EF93FF93B6
:10191000E6E4F0E00E949D13FF91EF913A9531F7D4
:101920009923E1F680E0809311013A9A3B9A43981B
:10193000A1E1B1E0119698E08E91983018F4392F1A
:10194000992702C038E09850881F429808F4429ABC
:1019500000000000439AEF93FF93E6E4F0E00E945A
:101960009D13FF91EF914398EF93FF93E6E4F0E02E
:101970000E949D13FF91EF913A9531F79923E1F67B
:1019800080E2809311013A9A3B9A4398A1E1B1E039
:10199000119698E08E91983018F4392F992702C04B
:1019A00038E09850881F429808F4429A00000000DE
:1019B000439AEF93FF93E6E4F0E00E949D13FF91BA
:1019C000EF914398EF93FF93E6E4F0E00E949D13BC
:1019D000FF91EF913A9531F79923E1F6419A4198B9
:1019E0003A9A3B9A4398A2E0B1E0119698E08E9122
:1019F000983018F4392F992702C038E09850881F82
:101A0000429808F4429A00000000439AEF93FF9333
:101A1000E6E4F0E00E949D13FF91EF914398EF936D
:101A2000FF93E6E4F0E00E949D13FF91EF913A9559
:101A300031F79923E1F680EC80930C013A9A3B9AB6
:101A40004398ACE0B1E0119698E08E91983018F48C
:101A5000392F992702C038E09850881F429808F41F
:101A6000429A00000000439AEF93FF93E6E4F0E00F
:101A70000E949D13FF91EF914398EF93FF93E6E44B
:101A8000F0E00E949D13FF91EF913A9531F7992371
:101A9000E1F63A9A3B9A4398A4E1B1E0119698E0B6
:101AA0008E91983018F4392F992702C038E0985059
:101AB000881F429808F4429A00000000439AEF936E
:101AC000FF93E6E4F0E00E949D13FF91EF914398AD
:101AD000EF93FF93E6E4F0E00E949D13FF91EF91F6
:101AE0003A9531F79923E1F680E0809315013A9A0F
:101AF0003B9A4398A5E1B1E0119698E08E91983019
:101B000018F4392F992702C038E09850881F42985E
:101B100008F4429A00000000439AEF93FF93E6E432
:101B2000F0E00E949D13FF91EF914398EF93FF9394
:101B3000E6E4F0E00E949D13FF91EF913A9531F7B2
:101B40009923E1F68091E004809315013A9A3B9A3B
:101B50004398A5E1B1E0119698E08E91983018F481
:101B6000392F992702C038E09850881F429808F40E
:101B7000429A00000000439AEF93FF93E6E4F0E0FE
:101B80000E949D13FF91EF914398EF93FF93E6E43A
:101B9000F0E00E949D13FF91EF913A9531F7992360
:101BA000E1F680E2809315013A9A3B9A4398A5E1C9
:101BB000B1E0119698E08E91983018F4392F99275A
:101BC00002C038E09850881F429808F4429A0000FA
:101BD0000000439AEF93FF93E6E4F0E00E949D1328
:101BE000FF91EF914398EF93FF93E6E4F0E00E94BA
:101BF0009D13FF91EF913A9531F79923E1F6419AC0
:101C000081E090E00E94A61341983A9A3B9A43984B
:101C1000A2E0B1E0119698E08E91983018F4392F37
:101C2000992702C038E09850881F429808F4429AD9
:101C300000000000439A00000000439800000000EC
:101C40003A9591F7992341F780E880930C013A9AED
:101C50003B9A4398ACE0B1E0119698E08E919830B1
:101C600018F4392F992702C038E09850881F4298FD
:101C700008F4429A00000000439AEF93FF93E6E4D1
:101C8000F0E00E949D13FF91EF914398EF93FF9333
:101C9000E6E4F0E00E949D13FF91EF913A9531F751
:101CA0009923E1F63A9A3B9A4398A1E0B1E0119664
:101CB00098E08E91983018F4392F992702C038E0B7
:101CC0009850881F429808F4429A00000000439AF6
:101CD000EF93FF93E6E4F0E00E949D13FF91EF91F4
:101CE0004398EF93FF93E6E4F0E00E949D13FF9189
:101CF000EF913A9531F79923E1F63A9A3B9A439856
:101D0000A6EDB4E0149690E28E91983018F4392F35
:101D1000992702C038E09850881F429808F4429AE8
:101D200000000000439AEF93FF93E6E4F0E00E9486
:101D30009D13FF91EF914398EF93FF93E6E4F0E05A
:101D40000E949D13FF91EF913A9531F79923E1F6A7
:101D50003A9A3B9A4398A2E0B1E0119698E08E91AE
:101D6000983018F4392F992702C038E09850881F0E
:101D7000429808F4429A00000000439A00000000D4
:101D80004398000000003A9591F7992341F780E4C9
:101D900080930C013A9A3B9A4398ACE0B1E01196DB
:101DA00098E08E91983018F4392F992702C038E0C6
:101DB0009850881F429808F4429A00000000439A05
:101DC000EF93FF93E6E4F0E00E949D13FF91EF9103
:101DD0004398EF93FF93E6E4F0E00E949D13FF9198
:101DE000EF913A9531F79923E1F63A9A3B9A439865
:101DF000A1E0B1E0119698E08E91983018F4392F57
:101E0000992702C038E09850881F429808F4429AF7
:101E100000000000439AEF93FF93E6E4F0E00E9495
:101E20009D13FF91EF914398EF93FF93E6E4F0E069
:101E30000E949D13FF91EF913A9531F79923E1F6B6
:101E40003A9A3B9A4398AAEDB4E0149690E28E91A8
:101E5000983018F4392F992702C038E09850881F1D
:101E6000429808F4429A00000000439AEF93FF93CF
:101E7000E6E4F0E00E949D13FF91EF914398EF9309
:101E8000FF93E6E4F0E00E949D13FF91EF913A95F5
:101E900031F79923E1F63A9A3B9A4398A2E0B1E0F0
:101EA000119698E08E91983018F4392F992702C036
:101EB00038E09850881F429808F4429A00000000C9
:101EC000439AEF93FF93E6E4F0E00E949D13FF91A5
:101ED000EF914398EF93FF93E6E4F0E00E949D13A7
:101EE000FF91EF913A9531F79923E1F680EC8093D9
:101EF0000C013A9A3B9A4398ACE0B1E0119698E015
:101F00008E91983018F4392F992702C038E09850F4
:101F1000881F429808F4429A00000000439AEF9309
:101F2000FF93E6E4F0E00E949D13FF91EF91439848
:101F3000EF93FF93E6E4F0E00E949D13FF91EF9191
:101F40003A9531F79923E1F680E090E0A5EEB4E010
:101F50008D939C933A9A3B9A4398A3E0B1E01196F3
:101F600098E08E91983018F4392F992702C038E004
:101F70009850881F429808F4429A00000000439A43
:101F8000EF93FF93E6E4F0E00E949D13FF91EF9141
:101F90004398EF93FF93E6E4F0E00E949D13FF91D6
:101FA000EF913A9531F79923E1F63A9A3B9A4398A3
:101FB000A5EEB4E0129690E18E91983018F4392F86
:101FC000992702C038E09850881F429808F4429A36
:101FD00000000000439AEF93FF93E6E4F0E00E94D4
:101FE0009D13FF91EF914398EF93FF93E6E4F0E0A8
:101FF0000E949D13FF91EF913A9531F79923E1F6F5
:102000003A9A3B9A4398A2E0B1E0119698E08E91FB
:10201000983018F4392F992702C038E09850881F5B
:10202000429808F4429A00000000439AEF93FF930D
:10203000E6E4F0E00E949D13FF91EF914398EF9347
:10204000FF93E6E4F0E00E949D13FF91EF913A9533
:1020500031F79923E1F680E480930C013A9A3B9A98
:102060004398ACE0B1E0119698E08E91983018F466
:10207000392F992702C038E09850881F429808F4F9
:10208000429A00000000439AEF93FF93E6E4F0E0E9
:102090000E949D13FF91EF914398EF93FF93E6E425
:1020A000F0E00E949D13FF91EF913A9531F799234B
:1020B000E1F63A9A3B9A4398A3E0B1E0119698E092
:1020C0008E91983018F4392F992702C038E0985033
:1020D000881F429808F4429A00000000439AEF9348
:1020E000FF93E6E4F0E00E949D13FF91EF91439887
:1020F000EF93FF93E6E4F0E00E949D13FF91EF91D0
:102100003A9531F79923E1F63A9A3B9A4398AEED26
:10211000B4E0129690E18E91983018F4392F9927F7
:1021200002C038E09850881F429808F4429A000094
:102130000000439AEF93FF93E6E4F0E00E949D13C2
:10214000FF91EF914398EF93FF93E6E4F0E00E9454
:102150009D13FF91EF913A9531F79923E1F6419A5A
:1021600081E090E00E94A61341988091E104809361
:10217000E80486E08093E9048091E1048093E80418
:102180003A9A3B9A4398A2E0B1E0119698E08E917A
:10219000983018F4392F992702C038E09850881FDA
:1021A000429808F4429A00000000439AEF93FF938C
:1021B000E6E4F0E00E949D13FF91EF914398EF93C6
:1021C000FF93E6E4F0E00E949D13FF91EF913A95B2
:1021D00031F79923E1F680E480930C013A9A3B9A17
:1021E0004398ACE0B1E0119698E08E91983018F4E5
:1021F000392F992702C038E09850881F429808F478
:10220000429A00000000439AEF93FF93E6E4F0E067
:102210000E949D13FF91EF914398EF93FF93E6E4A3
:10222000F0E00E949D13FF91EF913A9531F79923C9
:10223000E1F63A9A3B9A4398A9EEB4E0119698E0F9
:102240008E91983018F4392F992702C038E09850B1
:10225000881F429808F4429A00000000439AEF93C6
:10226000FF93E6E4F0E00E949D13FF91EF91439805
:10227000EF93FF93E6E4F0E00E949D13FF91EF914E
:102280003A9531F79923E1F680E08093E7043A9A92
:102290003B9A4398A7EEB4E0119698E08E9198305F
:1022A00018F4392F992702C038E09850881F4298B7
:1022B00008F4429A00000000439AEF93FF93E6E48B
:1022C000F0E00E949D13FF91EF914398EF93FF93ED
:1022D000E6E4F0E00E949D13FF91EF913A9531F70B
:1022E0009923E1F698E0A1EEB4E00E94EF1300918B
:1022F000E10440E1040FA7EEB4E00C933A9A3B9A54
:102300004398A7EEB4E0119698E08E91983018F4B7
:10231000392F992702C038E09850881F429808F456
:10232000429A00000000439AEF93FF93E6E4F0E046
:102330000E949D13FF91EF914398EF93FF93E6E482
:10234000F0E00E949D13FF91EF913A9531F79923A8
:10235000E1F63A9A3B9A4398A8EEB4E0119698E0D9
:102360008E91983018F4392F992702C038E0985090
:10237000881F429808F4429A00000000439AEF93A5
:10238000FF93E6E4F0E00E949D13FF91EF914398E4
:10239000EF93FF93E6E4F0E00E949D13FF91EF912D
:1023A0003A9531F79923E1F6419A81E090E00E9455
:1023B000A61341988091E3048093E8043A9A3B9AEB
:1023C0004398A2E0B1E0119698E08E91983018F40D
:1023D000392F992702C038E09850881F429808F496
:1023E000429A00000000439AEF93FF93E6E4F0E086
:1023F0000E949D13FF91EF914398EF93FF93E6E4C2
:10240000F0E00E949D13FF91EF913A9531F79923E7
:10241000E1F680E880930C013A9A3B9A4398ACE04D
:10242000B1E0119698E08E91983018F4392F9927E1
:1024300002C038E09850881F429808F4429A000081
:102440000000439AEF93FF93E6E4F0E00E949D13AF
:10245000FF91EF914398EF93FF93E6E4F0E00E9441
:102460009D13FF91EF913A9531F79923E1F63A9A4E
:102470003B9A4398A9EEB4E0119698E08E9198307B
:1024800018F4392F992702C038E09850881F4298D5
:1024900008F4429A00000000439AEF93FF93E6E4A9
:1024A000F0E00E949D13FF91EF914398EF93FF930B
:1024B000E6E4F0E00E949D13FF91EF913A9531F729
:1024C0009923E1F680E08093E7043A9A3B9A439897
:1024D000A7EEB4E0119698E08E91983018F4392F59
:1024E000992702C038E09850881F429808F4429A11
:1024F00000000000439AEF93FF93E6E4F0E00E94AF
:102500009D13FF91EF914398EF93FF93E6E4F0E082
:102510000E949D13FF91EF913A9531F79923E1F6CF
:1025200098E0A3EEB4E00E94EF130091E30440E1D1
:10253000040FA7EEB4E00C933A9A3B9A4398A7EEA7
:10254000B4E0119698E08E91983018F4392F9927BD
:1025500002C038E09850881F429808F4429A000060
:102560000000439AEF93FF93E6E4F0E00E949D138E
:10257000FF91EF914398EF93FF93E6E4F0E00E9420
:102580009D13FF91EF913A9531F79923E1F63A9A2D
:102590003B9A4398A8EEB4E0119698E08E9198305B
:1025A00018F4392F992702C038E09850881F4298B4
:1025B00008F4429A00000000439AEF93FF93E6E488
:1025C000F0E00E949D13FF91EF914398EF93FF93EA
:1025D000E6E4F0E00E949D13FF91EF913A9531F708
:1025E0009923E1F6419A81E090E00E94A613419878
:1025F00008950D911D912D913C9181E0080F882740
:10260000181F281F381F3C932E931E930E93089576
:10261000A8EBB0E118D0883091F08D3039F0332339
:10262000C9F38D933A9563FE24D0F4CF63FC04C0C4
:102630008DE01FD08AE01DD088278C93089519D093
:1026400011973395E7CF8091C00087FFFCCF809131
:10265000C60008950E94FA13802D11F00AD0FACF17
:1026600008958D9106D03A95E1F708958DE001D057
:102670008AE00090C00005FEFCCF8093C60008955C
:1026800088EE93E063D03197D9F7089500FC05D028
:10269000089530D005D001F8F9CF37D03FD0089554
:1026A000842F952FA62FB72FE894452B462B472B29
:1026B00011F468940895402F512F622F732F002733
:1026C000112722273327F0E2440F551F661F771F7B
:1026D000001F111F221F331F081B190B2A0B3B0B56
:1026E000416028F4080F191F2A1F3B1F4E7FFA95DF
:1026F00059F708950024E89477FF02C006D0689443
:1027000000F809D010F80124089512D04F5F5F4FF0
:102710006F4F7F4F0895E89437FF08950095109507
:10272000209530950F5F1F4F2F4F3F4F68940895AE
:10273000409550956095709508953197F1F70895FB
:10274000689462F80895E89462F80895EF93FF930F
:10275000EE27E82BE92B31F0E6E6FEE03197F1F7C2
:102760000197D1F7FF91EF9108950F921F922F9249
:10277000C801D901489F80014A9F90014B9F202C9E
:10278000499F100D211D321D5A9F202C589F100D5E
:10279000211D321D599F200D311D689F200D311DB7
:1027A000699F300D789F300D2F901F900F900895E6
:1027B00070917A00706470937A0000907A0006FC41
:1027C000FCCF70917A00706470937A0000907A0068
:1027D00006FCFCCF809178009091790008959030AC
:1027E00041F00D911C91169507959A95E1F71C9370
:1027F0000E930895C895319600200895040F151F73
:10280000261F371F08950417150726073707089551
:10281000000F111F221F331F08950095109520955A
:1028200030950F5F1F4F2F4F3F4F089500271127FF
:10283000222733271DD08A3328F4803318F005D09F
:1028400015D0F9CF0EF4E9CF089580538F93402F20
:10285000512F622F732FDCDFDBDFD0DFD9DF8F91C9
:102860009927080F191F291F391F08958D91089561
:10287000E894FCDF8032E9F38B32D9F38930C9F375
:102880008D3211F46894F2CF0895E89463F80895B6
:10289000689463F808954649524D57415245205671
:1028A000312E34342032322D30352D32303130005B
:00000001FF
